:060000000A128A11122809
:10000800FE00030EF7000408F8000A08F90083123E
:1000180003137F08FA000A128A11722D0A128A1134
:1000280015288313BE30FD000730FE003E30FF0068
:10003800AF3084000A128A1131270A128A11A030BF
:100048008400AF300A128A1159270A128A115330D4
:1000580084006B300A128A115927F001F101F2016C
:10006800F301F401F50183010A128A113B280A12EF
:100078008A11C0210A128A1157300A128A11E425FE
:100088000A128A1183120313C701C8018C12333074
:1000980083120313C600BB30C500DF30C400C40B95
:1000A8005328C50B5328C60B532883120313CB01BF
:1000B800CC018B170B17831603138C1683120313AB
:1000C800851E98284C08803AFF0080307F02031D67
:1000D8006F2802304B0203189828831203138814E0
:1000E800081537300A128A11E4250A128A111530C8
:1000F80083120313C6004B30C500BD30C400C40BC7
:100108008328C50B8328C60B83288A28AF300A1298
:100118008A1185260A128A11013083120313CB072C
:100128000318CC0A0030CC0783120313851A9E28C3
:100138008810081153035404031D5D28AF30A00034
:100148000030A100A0300A128A11B8260A128A11BA
:100158008312031320082104031D6929CA30A00053
:100168008030A10059300A128A11B8260A128A1161
:100178008312031320082104031DC52808108810C2
:100188000811D130A0008030A10059300A128A111C
:10019800B8260A128A118312031320082104031DAA
:1001A800EC280814CB01CC01333083120313C600AA
:1001B800BB30C500DF30C400C40BE028C50BE02805
:1001C800C60BE02884300A128A11E4250A128A1123
:1001D800BB3083120313A0008030A10059300A12EB
:1001E8008A11B8260A128A118312031320082104DF
:1001F800031D142988140815333083120313C6000D
:10020800BB30C500DF30C400C40B0829C50B082962
:10021800C60B082901300A128A11E4250A128A112C
:100228006330831203135906031D692968305A067F
:10023800031D69296E305B06031D69290030A8007B
:10024800A900AF300A128A11E7260A128A1183120E
:1002580003132108AB002008AA00AF300A128A1144
:100268000F270A128A11FF3083120313C900FF30C7
:10027800CA000330CD000030CE0059300A128A116E
:10028800E7260A128A118312031321084E02031D5E
:100298004F2920084D02031869290130C90703189E
:1002A800CA0A0030CA074D08593E84008313000863
:1002B800C4004908AF3E8400440880000130CD07DF
:1002C8000318CE0A0030CE0741290B3083120313DE
:1002D800C6002630C5005D30C400C40B7129C50BAB
:1002E8007129C60B712983120313D301D401F201BA
:1002F800F301F001F101CF01D0015008803AC400A8
:100308005808803A4402031D8B2957084F020318E6
:100318009B29831203134F08593E840083138001DD
:100328000130CF070318D00A0030D0078129831283
:100338000313D701D801D101D2015208803AC40071
:100348005608803A4402031DAB2955085102031888
:10035800BB29831203135108A03E84008313800134
:100368000130D1070318D20A0030D207A12983121D
:100378000313D501D6015D2883120313D701D801D1
:10038800D501D6010730C1004108831603139F0425
:100398009F111F159F141F1480308700FF308500A0
:1003A8008312031385128316031388018312031320
:1003B8000812881188128810081108140030B20039
:1003C8000030B1002530B0008030AF000A128A1129
:1003D800F4220A128A11153083120313C3004B301A
:1003E800C200BD30C100C10BF729C20BF729C30BEE
:1003F800F729FE2983120313081208160630831200
:100408000313C3001330C200AD30C100C10B0A2A68
:10041800C20B0A2AC30B0A2A831203130812663076
:1004280083120313C3007630C200C030C100C10B71
:100438001B2AC20B1B2AC30B1B2A0000CE308312B7
:100448000313A1008030A2000A128A1144260A125E
:100458008A110D300A128A114D270A128A110630A4
:1004680083120313C3001330C200AD30C100C10BA7
:100478003B2AC20B3B2AC30B3B2ACE308312031301
:10048800A1008030A2000A128A1144260A128A1199
:100498000D300A128A114D270A128A11063083126A
:1004A8000313C3001330C200AD30C100C10B5A2A78
:1004B800C20B5A2AC30B5A2AC13083120313A10054
:1004C8008030A2000A128A1144260A128A110D30BD
:1004D8000A128A114D270A128A1106308312031351
:1004E800C3001330C200AD30C100C10B792AC20B62
:1004F800792AC30B792A963083120313A10080301E
:10050800A2000A128A1144260A128A110D300A1210
:100518008A114D270A128A11063083120313C30069
:100528001330C200AD30C100C10B982AC20B982A03
:10053800C30B982A723083120313A1008030A200E3
:100548000A128A1144260A128A110D300A128A11D7
:100558004D270A128A110B3083120313C300263069
:10056800C2005D30C100C10BB72AC20BB72AC30B4A
:10057800B72AA03083120313A1008030A2000A1208
:100588008A1144260A128A1122300A128A114D272A
:100598000A128A11B33083120313A1008030A2001B
:1005A8000A128A1144260A128A1122300A128A1162
:1005B8004D270A128A110D300A128A114D270A1284
:1005C8008A110B3083120313C3002630C2005D303A
:1005D800C100C10BED2AC20BED2AC30BED2A08009E
:1005E800831203132F08B3003008B4003108B50094
:1005F8003208B60006300310B30DB40DB50DB60DB4
:10060800FF3E031DFF2A3608A3003508A200340860
:10061800A1003308A0000030B7001230B8007A30CB
:10062800B9000030BA002F08BB003008BC00310800
:10063800BD003208BE0006300310BB0DBC0DBD0D59
:10064800BE0DFF3E031D202BBB09BC09BD09BE0919
:10065800BB0A0319BC0A0319BD0A0319BE0A3B08E1
:10066800B7073C0803183C0F3A2B3B2BB8073D084B
:1006780003183D0F402B412BB9073E0803183E0ACB
:10068800BA073A08A7003908A6003808A5003708AD
:10069800A4000A128A11E3240A128A11831203138E
:1006A8002108C0002008BF000130400200300319B3
:1006B8003F02031CC42B2F08B3003008B4003108D4
:1006C800B5003208B60004300310B30DB40DB50DF3
:1006D800B60DFF3E031D682B3608A3003508A2009F
:1006E8003408A1003308A0000030B7001230B80069
:1006F8007A30B9000030BA002F08BB003008BC00BF
:100708003108BD003208BE0004300310BB0DBC0D1B
:10071800BD0DBE0DFF3E031D892BBB09BC09BD09DC
:10072800BE09BB0A0319BC0A0319BD0A0319BE0A8C
:100738003B08B7073C0803183C0FA32BA42BB807AA
:100748003D0803183D0FA92BAA2BB9073E0803182B
:100758003E0ABA073A08A7003908A6003808A500D3
:100768003708A4000A128A11E3240A128A11831294
:1007780003132108C0002008BF00831603131815AF
:10078800013083124002003003193F0203180800A9
:100798003F0883160313990018128312031398173E
:1007A80080308316031387008312031318168316E9
:0607B8000313981608006F
:10080000FF1B0A2C83137F1883170008840A03191F
:10081000FF0A080004308A000408840A82070034B2
:10082000483465342034743468346F346E3467343B
:100830002034623461346F34203464346F346E3465
:1008400067342034623461346E3467342034743455
:1008500069346E3420346E34683461346E3420343C
:1008600068346F3461347434203464346F346E34DB
:1008700067342034623469346E346834203474341C
:10088000683475346F346E346734003443346F34F5
:1008900020346334683461347934203478346134FA
:1008A00079342034723461342034743461346934DE
:1008B0002034703468346F346E3467342034373405
:1008C00030343634203445343334003448346534DD
:1008D0002034743468346F346E34673420346434B4
:1008E00061342034643475346F34633420346B34B1
:1008F00068346F346934203464346F346E34673450
:100900000034413454342B3443344E344D34493460
:100910003D3432342C3432342C3430342C343034B2
:100920002C34303400344834653420347434683422
:100930006F346E3467342034643475346F34633408
:1009400020346234613474340034413454342B34F0
:1009500043344D34473446343D343134003441342B
:1009600054342B3443344D344734443441343D34CF
:100970000034413454342B3443344D3447345334ED
:100980003D340034443445344C34203441344C3408
:100990004C34003463346834653463346B3400346D
:1009A00041345434453430340034413454344434C4
:1009B00000346F34663466340034413454340034C7
:1009C0006F346E34003483120313AA01A31FF52C75
:1009D000A009A109A209A309A00A0319A10A0319E0
:1009E000A20A0319A30AAA01AA0AA71F062DA4098D
:1009F000A509A609A709A40A0319A50A0319A60AA5
:100A00000319A70A0130A8002808AA060030AE0082
:100A10000030AD000030AC000030AB0023082204F1
:100A20002104200403195B2DA901A90AA31B262D6B
:100A30000130A8000310A00DA10DA20DA30DA80B5D
:100A40001A2D0130A8002808A907162D0130A8008A
:100A50000310AB0DAC0DAD0DAE0DA80B282D23086A
:100A60002702031D3D2D22082602031D3D2D2108CE
:100A70002502031D3D2D20082402031C4E2D2008B5
:100A8000A4022108031C210FA5022208031C220F27
:100A9000A6022308031C230FA7022B140130031006
:100AA000A30CA20CA10CA00CFF3E031D4F2D013086
:100AB000A902031D262D2A080319692DAB09AC09CB
:100AC000AD09AE09AB0A0319AC0A0319AD0A031943
:100AD000AE0A2E08A3002D08A2002C08A1002B08A6
:100AE000A00008008C1ED92D1A08F6007608FB001D
:100AF000023070067104031D8B2D0D307B06031D23
:100B00008B2D0130F0070318F10A0030F107013096
:100B1000D3000030D400023070067104031D9E2DF6
:100B20007B08F6005708593E84007608831380003E
:100B30000130D7070318D80A0030D8070A307B06DF
:100B4000031DA82D0130F0070318F10A0030F1074A
:100B500072037304031DB62D22307B06031DB62DD0
:100B60000130F2070318F30A0030F307720373042D
:100B7000031DC82D7B08F6005508A03E84007608AA
:100B8000831380000130D5070318D60A0030D6073A
:100B900022307B06031DD22D0130F2070318F30A21
:100BA0000030F307981CD92D18120000831203138C
:100BB00018167A08FF0079088A0078088400770EF2
:100BC0008300FE0E7E0E090083120313AB00AA30D1
:100BD000A1008030A2000A128A1144260A128A114A
:100BE00022300A128A114D270A128A11AF3083125D
:100BF0000313A1000030A2000A128A1144260A122F
:100C00008A1122300A128A114D270A128A110D30D8
:100C10000A128A114D270A128A110B30831203130C
:100C2000AA002630A9005D30A800A80B152EA90B3C
:100C3000152EAA0B152E831203132B08A1000030CA
:100C4000031D8030A2000A128A1144260A128A115A
:100C50000D300A128A114D270A128A111A300A120F
:100C60008A114D270A128A11153083120313AA0024
:100C70004B30A900BD30A800A80B3C2EA90B3C2E80
:100C8000AA0B3C2E432E080083120313A601A701D2
:100C900026082107A4002208A3000318A30AA61B04
:100CA000A303831203132308A5002508FF002408CB
:100CB00084000A128A1100240A128A11003A0319C8
:100CC000080026082107A4002208A3000318A30A8D
:100CD000A61BA303831203132308A5002508FF0006
:100CE000240884000A128A1100240A128A110A12A6
:100CF0008A114D270A128A11013083120313A607A5
:100D00000318A70A0030A707482E83120313AB006D
:100D1000C630A1008030A2000A128A1144260A12AD
:100D20008A11831203132B08A1000030A2000A12BB
:100D30008A1144260A128A113B300A128A114D2761
:100D40000A128A110D300A128A114D270A128A11CD
:100D5000CB3083120313AA00EC30A9008330A80023
:100D6000A80BB02EA90BB02EAA0BB02EB72E0800E0
:100D700083120313A500C42E0130A2002208A50788
:100D80000130A0070318A10A250884008313000876
:100D9000A2002108FF00200884000A128A11002402
:100DA0000A128A11FF3A013E2207A3002308A40079
:100DB0002408031DE12E2508840083130008031D69
:100DC000BC2E2408A000A101A01BA10308008312CF
:100DD0000313A6002608A2002208A7002708840003
:100DE000831300080319F92E0130A2002208A70777
:100DF000EE2E2608A2000030A300A209A309A20A31
:100E00000319A30A2708A4000030A500220824071C
:100E1000A00023080318230A2507A1000800831255
:100E20000313AD002D08AC002C08AE000130AA025F
:100E30000030031CAB03AB022A0A03192B0A031967
:100E400008002808AC002E0884002C0883138000BA
:100E50000130AC002C08AE07162F7E088A007F08F0
:100E600082002D270A128A118000840A04087D0658
:100E700003190034FF0A0319FE0A312F2B343834CA
:100E80003434333433343534353430343634323426
:100E90003834393400340034003483120313A00092
:100EA00083160313981C502F8312031320089900F4
:100EB000080064008001840A040603190034040653
:020EC0005A2FA7
:02400E003A3F37
:00000001FF
